:1000000000308A003E280000831685108312851078
:1000100008308D000000000000008D171F288D1390
:10002000900C03188514031C85100D171F280D1341
:100030008D0B102800000000000085141F281C30C4
:100040008400840B212800008D1B0F280D1B17280E
:100050004A2811308400000803193D2801308D0022
:100060008C018C0B31288D0B30284A308C008C0B86
:10007000372800000000800B2E284F2884011F30F5
:100080008305831685108312851441308F000F0875
:100090009000042804309000FA3091002928900B39
:1000A0004C288F0A0F087A3C03184728452863001C
:00000001FF
